:020000020000FC
:100000000DC0189518951895189518951895189568
:10001000ABC01895189518951895CAC000E00EBF8A
:100020000FED0DBF00E808B901E007B907EC06B90C
:1000300002E001B903E00EBD0DEF0DBD0FE80CBDF0
:1000400001E00CB94FEE00EF0ABB0BBB07E007BBAA
:10005000DD27C4E000E3402E502E602E702E7894F1
:10006000EE24FF2420E4339A49D097FF03C09F7702
:10007000369AFACF2223C1F73398F694E794F69490
:10008000E794F694E794E0E6F0E0E192F19253957C
:10009000583008F05527E0E6F0E0FF24EE24222750
:1000A0000191E00E0191F01E23952830C8F3F694DB
:1000B000E794F694E794F694E79404E713E12ED0DE
:1000C000269417942694179426941794F22CE12CD6
:1000D00032D0A4E0BB27022D0F70002319F40FEFDC
:1000E0000D9301C011D0012D029590640DD09F7B1E
:1000F000012D0AD0002D029507D0B2CF00E205BF36
:100100008895002705BF0895ECEBF1E00F70E00F34
:10011000FB1F049196FD0F7D0D930895222420E18D
:100120001695079510F41E0C2F1C2794179407940E
:100130002A95B1F7089520E1222411240024FF27F5
:10014000EE0CFF1C001C111C221C2A9509F40895BA
:10015000E3E002910D5F03FD00830081005D07FD78
:100160000083E030B1F7ECCF0F930FB70F930DEF93
:100170000DBD0FE80CBD0BB3006F0BBBC29809910E
:1001800038E0C098000F10F4C19A01C0C198C09A1D
:100190003A95B9F7C29A0BB3006F04230BBB440F17
:1001A00010F04FEEC4E090680F910FBF0F911895BB
:1001B00004B1E00E05B1F01E2A95189530F32AA27D
:0601C000E1A424F220A0DE
:00000001FF
